:060000009031232B0000EB
:0800080083018031200077081C
:10001000A0007808A1007908A2007A08A300850151
:1000200091308400801C162891181F282008F700A2
:100030002108F8002208F9002308FA000900883195
:1000400000280B003F3406345B344F3466346D3483
:100050007D3407347F346F3477347C3458345E34E5
:10006000793471342200A0012008013C031C6B2864
:10007000200821006C072200A400003021006D3D03
:100080002200A5002030A7009E30A60020082607E9
:10009000F8000030273DFA00780884007A088500CF
:1000A0000008A6000B08F7008B132408230091001A
:1000B000220026082300930095131515553096004D
:1000C000AA309600951495186328151177088B04AB
:1000D0002200A00A34282000080022000D128D12F0
:1000E0008C012100ED01EC01200051082100EF00FE
:1000F000200050082100EE00200032202100ED01F8
:100100000230EC00200053082100EF0020005208CC
:100110002100EE00200032202100ED010430EC002F
:10012000200055082100EF00200054082100EE00B7
:10013000200032202100ED010630EC00200057089D
:100140002100EF00200056082100EE0020003220A0
:100150002100ED010830EC00200059082100EF00DB
:10016000200058082100EE00200032202100ED017F
:100170000A30EC0020005B082100EF0020005A0844
:100180002100EE00200032202100ED010C30EC00B7
:1001900020005D082100EF0020005C082100EE0037
:1001A000200032200B08F7008B130E302300910043
:1001B00020005E0823009300951315155530960016
:1001C000AA30960095149518E328151177088B042A
:1001D000003020002E1901302100EC000B08F70040
:1001E0008B130F302300910021006C082300930033
:1001F0009513151555309600AA309600951495184C
:10020000FF28151177088B040B08F7008B131030AB
:10021000910020005F0823009300951315155530B9
:100220009600AA3096009514951814291511770890
:100230008B040B08F7008B1311309100200060082D
:10024000230093009513151555309600AA3096009B
:10025000951495182929151177088B040B08F700B8
:100260008B13123091002000610823009300951336
:10027000151555309600AA309600951495183E290C
:10028000151177088B04200008002508D43E0318B8
:10029000632D2C3E6F2D2C08FC3E03188D29043E47
:1002A000672D0230A5008D290330A5008D295C083B
:1002B000D0025D08D13BD11B6429D108031D6729F9
:1002C0005008633C031C6729D1016430D0005108F9
:1002D000E3005008E2000430F300B230F2008D2950
:1002E0005C08D0075D08D13DD11B85295108003C31
:1002F00003188529FF3A031D81295008C23C0318C1
:1003000085290130D100C230D0005108E3005008E7
:10031000E2000430F300B230F200632DD101D001CD
:100320002E1C9629AE1896290230AC00AE102E185D
:10033000AE142C08023A0319A129013A0319AC2979
:10034000B229A5016308D1006208D000EF01EE01D7
:10035000ED01EC01F001B2290330A5006308D100E2
:100360006208D000632DD31FB829D11FC429BA2930
:10037000D11BC82953085102031CC829031DC429D5
:10038000500852020318C8295308D1005208D0005F
:10039000E1080319D3297B086102031CD7297E08D1
:1003A0006102031CD7292E1CD929AE18D929023085
:1003B000AC00AE102E18AE142C08023A0319E42932
:1003C000013A0319FC29022AA5016308D100620839
:1003D000D000EF01EE01ED01EC01F001D408031DA6
:1003E000FB29D508031DFB29FF30EF00EE00E830A4
:1003F000ED008630EC00022A0330A5006308D1002E
:100400006208D000632D2C08023A03190E2A023A22
:100410000319102A013A0319132A152AA501152ACE
:100420001030A500152A0430A500632D2C08023ACF
:100430000319212A023A0319242A013A0319272A07
:10044000292A0530A500292A0330A500292A0630CB
:10045000A500632D2C08023A0319352A023A031924
:10046000392A013A0319472A572A6D200430A5007A
:10047000572AD31B462AD308031D422A5208643C3C
:100480000318462A0A30D2020030D33B572AD31B26
:10049000532A5308013C031C572A031D532A5208B0
:1004A000C13C031C572A0A30D2070030D33D632DCC
:1004B0002C08023A0319632A023A0319662A013A00
:1004C0000319692A6B2A0730A5006B2A0430A5009E
:1004D0006B2A0830A500632D2C08023A0319772AED
:1004E000023A03197B2A013A0319892A952A6D20B9
:1004F0000630A500952AD51B882AD508031D842A15
:100500005408003C0318882A54080319D503D4035F
:10051000952AD51B922AD508031D952A54081E3CFE
:10052000031C952AD40A0319D50A632D2C08023A14
:100530000319A12A023A0319A42A013A0319A72A86
:10054000A92A0930A500A92A0630A500A92A0A303F
:10055000A500632D2C08023A0319B52A023A0319A3
:10056000B92A013A0319C22AD22A6D200830A500FF
:10057000D22A0A30D6020030D73BD71FC12AD70172
:10058000D601D22A0A30D6070030D73DD71BD22A4F
:10059000D708031DCF2A5608783C0318D22AD70162
:1005A0008230D600632D2C08023A0319DE2A023A63
:1005B0000319E12A013A0319E42AE62A0B30A500BF
:1005C000E62A0830A500E62A0C30A500632D2C0889
:1005D000023A0319F22A023A0319F62A013A0319D8
:1005E000082B142B6D200A30A500142BD91F032BC8
:1005F0005908FE3C0318072BFF3A031D032B58082C
:10060000D83C0318072B58080319D903D803142B17
:10061000D91B112BD908031D142B5808273C031C88
:10062000142BD80A0319D90A632D2C08023A03198E
:10063000202B023A0319232B013A0319262B282BCE
:100640000D30A500282B0A30A500282B0E30A50060
:10065000632D2C08023A0319342B023A0319382B64
:10066000013A0319382B3F2B6D200C30A5003F2B8E
:10067000DE08031D3E2B0130DE003F2BDE01632D23
:100680002C08023A03194B2B023A03194E2B013A5C
:100690000319512B532B0F30A500532B0C30A50001
:1006A000532B1030A500632D2C08023A03195F2B41
:1006B000023A0319632B013A0319632B712B6D2046
:1006C0000E30A500712B5C08053C031D6E2BDD0868
:1006D000031D6E2BDD010130DC00712BDD010530C7
:1006E000DC00632D2C08023A03197D2B023A031912
:1006F000802B013A0319832B852B1130A500852B04
:100700000E30A500852B0330A500632D2C08023A7E
:100710000319912B023A0319942B013A0319972BD1
:10072000992B1030A500992B2A30A500992B123057
:10073000A500632D2C08023A0319A52B023A0319D0
:10074000A82B013A0319AB2BAD2B1330A500AD2B11
:100750001130A500AD2B1430A500632D2C08023AF2
:10076000031DB42B1230A500632D2C08023A031987
:10077000C02B023A0319C32B013A0319C62BC82B0D
:100780001530A500C82B1230A500C82B1630A500C7
:10079000632D2C08023A0319D42B023A0319D82BE3
:1007A000013A0319EA2BF92B6D201430A500F92B1F
:1007B000DB1BE92B5B08063C0318E92BFF3A031D02
:1007C000E52B5A08993C0318E92B5A080319DB0357
:1007D000DA03F92BDB1BF62B5B08083C031CF92B17
:1007E000031DF62B5A08663C031CF92BDA0A031981
:1007F000DB0A632D2C08023A0319052C023A03196F
:10080000082C013A03190B2C0D2C1730A5000D2CC8
:100810001430A5000D2C1830A500632D2C08023AC9
:10082000031D142C1630A500632D2C08023A031961
:10083000202C023A0319232C013A0319262C282CC8
:100840001930A500282C1630A500282C1A30A50038
:10085000632D2C08023A031D2F2C1830A500632DA0
:100860002C08023A03193B2C023A03193E2C013A98
:100870000319412C432C1B30A500432C1830A50034
:10088000432C1C30A500632D2C08023A031D4A2C72
:100890001A30A500632D2C08023A0319562C023A8F
:1008A0000319592C013A03195C2C5E2C1D30A5004C
:1008B0005E2C1A30A5005E2C1E30A500632D2C087E
:1008C000023A031D652C1C30A500632D2C08023A4A
:1008D0000319712C023A0319742C013A0319772C6D
:1008E000792C1F30A500792C1C30A500792C2030E4
:1008F000A500632D2C08023A031D802C1E30A50094
:10090000632D2C08023A03198C2C023A03198F2C00
:10091000013A0319922C942C2130A500942C1E30FE
:10092000A500942C2230A500632D2C08023A031D4B
:100930009B2C2030A500632D2C08023A0319A72C0C
:10094000023A0319AA2C013A0319AD2CAF2C23301B
:10095000A500AF2C2030A500AF2C2430A500632DBE
:100960002C08023A0319BB2C023A0319BF2C013A96
:100970000319C32CC72C6D202230A500C72CE10819
:10098000031DE103C72C61084A3C0318E10A632DEB
:100990002C08023A0319D32C023A0319D62C013A37
:1009A0000319D92CDB2C2530A500DB2C2230A50027
:1009B000DB2C2630A500632D2C08023A0319E72C06
:1009C000023A0319EB2C013A0319F02CF42C6D2098
:1009D0002430A500F42C6008083C0318E00AF42C2D
:1009E0006008033C031CE003632D2C08023A031942
:1009F000002D023A0319032D013A0319062D082D83
:100A00002730A500082D2430A500082D2830A5008A
:100A1000632D2C08023A0319142D023A0319182DDC
:100A2000013A0319182D1A2D6D202630A5001A2D14
:100A30000430AE06632D2C08023A0319262D023A23
:100A40000319292D013A03192C2D2E2D2930A5002B
:100A50002E2D2630A5002E2D2A30A500632D2C0822
:100A6000023A03193A2D023A03193E2D013A0319AD
:100A70003E2D472D6D202830A500472D5F08323CC4
:100A8000031D452D3C30DF00472D3230DF00632D44
:100A90002C08023A0319532D023A0319562D013A34
:100AA0000319592D5B2D2B30A5005B2D2830A50097
:100AB0005B2D1130A500632D2C08023A031D622D19
:100AC0002A30A500632D0430AC0088312B2A0A148B
:100AD0008A100A15820757297029512954290A14A6
:100AE0008A100A1582074B29B3298E29032A162A50
:100AF0002A2A582A6C2A962AAA2AD32AE72A152BA8
:100B0000292B402B542B722B862B9A2BAE2BB52BDB
:100B1000C92BFA2B0E2C152C292C302C442C4B2CA9
:100B20005F2C662C7A2C812C952C9C2CB02CC82CFC
:100B3000DC2CF52C092D1B2D2F2D482D5C2D210093
:100B4000C6014608013C031CC32D2030CD00773080
:100B5000CC0046084C07F80000304D3DFA007808FC
:100B600084007A08850046084407CE000030453DE1
:100B7000CF004E0823009100951315141308800030
:100B80002100C60AA12D4708F8004808F9002000F6
:100B900008000430F80021001D08833978049D0006
:100BA0000F30F8001F08F03978049F0022008D16DE
:100BB0003530F700F70BDA2D21009D149D18DE2D3E
:100BC0001C08C5001B08C40022008D122100450826
:100BD0000E3C0318F62DFF3A031DF22D4408A03CED
:100BE0000318F62D01302000AD0021002000080080
:100BF0002030850074308400000803190C2E0A3060
:100C0000F800F701F70B022EF80B012E5F30F7000A
:100C1000F70B082E800BFF2D9031442D2100460D3F
:100C2000F700F70DFC30F7051D08833977049D00A8
:100C30000F30F8001F08F03978049F000D30F700DE
:100C4000F70B202E2000E401C701C60164080F3C09
:100C5000031C372E21009D149D182C2E1C08FA0011
:100C60001B082000C6077A08C73DE40A262E21008B
:100C70004408840045088500200046088000470895
:100C8000813F080021005208F70003102300951748
:100C9000151400000000130880000131910A0319A7
:100CA000920AF70B482E2000080020302100E000B7
:100CB000DC01DD01DE01DF015508FA005408F9000E
:100CC0005308F8005208F7000310771C752E5608D9
:100CD000DC0757080318570FDD0758080318580F8B
:100CE000DE0759080318590FDF07DF0CDE0CDD0C97
:100CF000DC0CFA0CF90CF80CF70CE00B642E20005D
:100D000008008318872E2030850088308400210059
:100D10004F0853068039DD00CF1F992ECC09CD092D
:100D2000CE09CF09CC0A0319CD0A0319CE0A03193B
:100D3000CF0AD31FA62ED009D109D209D309D00AD0
:100D40000319D10A0319D20A0319D30AF701F801CA
:100D5000F901FA01D801D901DA01DB015308520483
:100D6000510450040319E42E2030DC000310CC0D94
:100D7000CD0DCE0DCF0DD80DD90DDA0DDB0D5308ED
:100D80005B02031DCD2E52085A02031DCD2E5108C1
:100D90005902031DCD2E50085802031CDE2E5008A8
:100DA000D8025108031C510FD9025208031C520FDC
:100DB000DA025308031C530FDB020314F70DF80D7E
:100DC000F90DFA0DDC0BB62EDD1FF12EF709F8092F
:100DD000F909FA09F70A0319F80A0319F90A0319B4
:100DE000FA0A580880005908813F5A08823F5B0878
:100DF000833F2000080010302100D600F701FA01DF
:100E0000D30CD20C031C0A2F5408F7070318FA0A54
:100E10005508FA07FA0CF70CF90CF80CD60B002F52
:100E2000200008002100520854068039D700D21F44
:100E30001E2FD109D209D10A0319D20AD41F252F96
:100E4000D309D409D30A0319D40AF801F901F70127
:100E5000FA015408031D2F2F53080319492F10308E
:100E6000D6000310D10DD20DF70DFA0D54087A02F9
:100E7000031D3C2F53087702031C452F5308F7022C
:100E8000031CFA035408FA020314F80DF90DD60BEB
:100E9000312FD71F502FF809F909F80A0319F90A59
:100EA0002000080021004E0850068039D300CE1FD4
:100EB0005E2FCD09CE09CD0A0319CE0AD01F652FAA
:100EC000CF09D009CF0A0319D00A1030D200F70198
:100ED000FA01CE0CCD0C031C732F4F08F707031833
:100EE000FA0A5008FA07FA0CF70CF90CF80CD20BB6
:100EF000692FD31F802FF809F909F80A0319F90A95
:100F000020000800F801F901F701FA012100490861
:100F1000031D8D2F48080319A72F1030CA00031096
:100F2000C60DC70DF70DFA0D49087A02031D9A2F59
:100F300048087702031CA32F4808F702031CFA0392
:100F40004908FA020314F80DF90DCA0B8F2F20007F
:020F5000080097
:10100000F60A5F08323C031D0B287608173C0318CC
:101010000A28F60110287608133C03181028F60158
:10102000AE1D18282E1818282100A4011B28200006
:1010300034082100A40022008C0120002F0803198D
:101040003728013A03197228033A0319AF28013AE5
:101050000319E928073A03191429013A03193C290D
:10106000033A03196429013A03199029CD29FE3066
:1010700022008E00210024080139F700EC017718C6
:10108000EC17200033080139F700F70EF70DF70DC4
:10109000C030F70577082100EC0420003208013940
:1010A000F700F70EF70DE030F70577082100EC04A4
:1010B000200031080139F700F70EF030F705770806
:1010C0002100EC04200030080139F700F70DF70D7E
:1010D000F70DF830F70577082100EC046C082200C2
:1010E0008C00D029FD3022008E0021002408023916
:1010F000F700770EEC00EC0DEC0DC030EC05200095
:1011000033080239F700F70EF70DE030F7057708DE
:101110002100EC04200032080239F700F70EF0300D
:10112000F70577082100EC04200031080239F700A8
:10113000F70DF70DF70DF830F70577082100EC04EF
:10114000200030080239F700F70DF70DFC30F705E5
:1011500077082100EC046C0822008C00D029FB30B9
:1011600022008E00210024080439F700770EEC00DD
:10117000EC0DE030EC05200033080439F700F70EE1
:10118000F030F70577082100EC042000320804391C
:10119000F700F70DF70DF70DF830F7057708210088
:1011A000EC04200031080439F700F70DF70DFC308E
:1011B000F70577082100EC04200030080439F70017
:1011C0000310F70D77082100EC046C0822008C0056
:1011D000D029F73022008E00200033080839F700AC
:1011E000770D2100EC00EC0DEC0DF830EC05200043
:1011F00032080839F700F70DF70DFC30F7057708CE
:101200002100EC04200031080839F7000310F70D25
:1012100077082100EC042000300808392100EC0494
:101220006C0822008C00D029EF3022008E002000B4
:1012300033081039F700770D2100EC00EC0DFC307D
:10124000EC05200032081039F7000310F70D77087D
:101250002100EC042000310810392100EC042000AA
:1012600030081039F7000310F70C77082100EC0460
:101270006C0822008C00D029DF3022008E00200074
:1012800033082039F7000310770D2100EC0020000F
:10129000320820392100EC04200031082039F70001
:1012A0000310F70C77082100EC04200030082039E7
:1012B000F700F70CF70C3F30F70577082100EC0436
:1012C0006C0822008C00D029BF3022008E00200044
:1012D000330840392100EC00200032084039F70083
:1012E0000310F70C77082100EC0420003108403986
:1012F000F700F70CF70C3F30F70577082100EC04F6
:10130000200030084039F700F70CF70CF70C1F30BD
:10131000F70577082100EC046C0822008C00D02926
:101320007F3022008E002000330880392100EC003D
:1013300020006A08FF3A21006C04F7000310770CC4
:10134000EC002000320880392100ED0020006B08FD
:10135000FF3A21006D04F700F70CF70C3F30F7055A
:101360007708EC04200031088039F700F70CF70CFF
:10137000F70C1F30F70577082100EC042000300837
:101380008039F700F70E0F30F70577082100EC04DD
:101390006C0822008C00D0292000FF3022008E0033
:1013A0002000AF0A2F08083C031DDD292508023C58
:1013B0000319DD29AF010830AE062F08103C031DCC
:1013C000E229AF018D1BEF290D1BE929351FE92902
:1013D000AC010D1FEF29351BEF290130AC000D08C2
:1013E000B500901D002AE808031DF929E908031932
:1013F000042AE908031D042A6808473C031C042A40
:10140000E80A0319E90A062AE901E801901D0D2AF4
:10141000E50803190D2AE503182A9019182AE90886
:10142000031D162A6808013C0318182A2430E50019
:10143000680B232AE908031D232AE508031D232A34
:101440000230AC00292A6908033C0318292A03301A
:10145000AC0080314529883161087B020318342AA9
:1014600061087E02031C362A2E18442AA508031997
:101470003B2A250B442A0130EC070318ED0A031917
:10148000EE0A0319EF0A492AEF01EE01ED01EC0122
:10149000F0016C0F5C2A6D08193C031D5C2A6E0B71
:1014A0005C2AEF08031D5C2AEF01EE01ED01EC015F
:1014B000700F5B2A5C2AF00A6C0B7A2AED08031D78
:1014C0007A2AEE08031D7A2AEF08031D7A2A5408A7
:1014D0007002031D7A2AD508031D7A2A54081F3C7E
:1014E000031D752AD50803197A2AA508031D7A2A2F
:1014F0000130A5006C0B9A2AED08031D9A2AEE080C
:10150000031D9A2AEF08031D9A2A56087002031D2C
:101510009A2AD708031D9A2A5608823C031D932A4B
:10152000D70803199A2AA5080319982A250B9A2A7D
:101530000230A500F208031DA02AF3080319A42A0B
:1015400072080319F303F203720BAB2AF308031DAD
:10155000AB2A0130F1006A087F3C031DB22AFC0A65
:101560000319FD0A6B087F3C031DBB2A2100A00A5A
:101570000319A10A20002100A20A0319A30A2208C4
:10158000203C031DE12A2308033C031DE12AA3019B
:10159000A2017D0CFA007C0CF900FA0CF90CFA0C93
:1015A000F90C7908FB00210CFA00200CF900FA0C68
:1015B000F90CFA0CF90C7908FE00FD01FC01A101FF
:1015C000A0012000911080311628E701E601E7080C
:1015D000031D2D2B6608143C031C2D2B21004508F0
:1015E000FA00440884007A0885000008CC00013124
:1015F0000008CD003F3103102000660DF900670D93
:10160000FA007908703E2100CE003F307A3DCF00CD
:101610004F082300920021004E0823009100203043
:1016200085008030840002302100D200803120000B
:101630004226883121004D085102031C282B031D2E
:10164000252B50084C020318282B20002D2B21009D
:101650002000E60A0319E70AE72A0310660DF900DD
:10166000670DFA007908703E2100CC003F307A3DCA
:10167000CD002300920021004C082300910020306F
:1016800085001E30840002302100D200803120000D
:1016900042268831013066022100CC000030200053
:1016A000673B2100CD0003104C0DF9004D0DFA00F1
:1016B0007908703ECC003F307A3DCD002300920087
:1016C00021004C0823009100203085002230840046
:1016D00002302100D20080312000422688312100D2
:1016E000440884004508850001310008FA003F31B4
:1016F000000820004202F7007A08433BF80000305F
:10170000443BF9000030453BFA002100CF00790846
:10171000CE007808CD007708CC000508D100040879
:10172000D000D501D401D3010A30D2004F08D9002E
:101730004E08D8004D08D7004C08D6008031200054
:1017400055268831210051088500500884007A0808
:101750002000B9007908B8007808B7007708B6000B
:101760003E084202F7003F08433BF8004008443B74
:10177000F9004108453BFA00BD007908BC00780833
:10178000BB007708BA00831039082100CF00200081
:1017900038082100CE00200037082100CD002000AD
:1017A00036082100CC0020003D082100D300200095
:1017B0003C082100D20020003B082100D10020007D
:1017C0003A082100D00080312000812688317A0833
:1017D0002100CF007908CE007808CD007708CC0032
:1017E000063020006602F7000030673BFA007708F9
:1017F0002100D0007A08D100D3010A30D20051086C
:10180000D5005008D40080312000FB2688317908AB
:10181000FA00780821004C07F70079084D3DF800E0
:1018200000304E3DF90000304F3DFA0078082000AE
:10183000CF007708CE0021004608840047088500C5
:1018400020004E0880004F08813F90314F2E21002C
:101850004508FA0044088400450885000008CC00CB
:1018600001310008CD0001310008CE00013100082F
:10187000CF003D3120005A08F7005B08F800F9015D
:10188000FA01DB1F452CF903FA0305082100D100FA
:101890000408D0004F08D5004E08D4004D08D300EE
:1018A0004C08D2007A08D9007908D8007808D70007
:1018B0007708D60080312000552688312100510854
:1018C0008500500884007A08CF007908CE00780897
:1018D000CD007708CC00CB014F0CCA004E0CC900DC
:1018E0004D0CC800CA0CC90CC80CCA0CC90CC80CD9
:1018F0001F30CA052000E701E601E708031DBB2CE5
:101900006608313C031CBB2C0310660DF900670D03
:10191000FA0079089A3E2100CC003F307A3DCD0094
:101920004D082300920021004C0823009100203034
:1019300085007E30840002302100D20080312000FA
:10194000422688312100CB08031DB62CCA08031D8E
:10195000B62C49084F02031CB62C031DB32C4E08AD
:1019600048020318B62C2000BB2C21002000E60AF8
:101970000319E70A7D2C0310660DF900670DFA00C4
:1019800079089A3E2100CC003F307A3DCD002300FB
:10199000920021004C0823009100203085001E3069
:1019A000840002302100D20080312000422688319C
:1019B000013066022100CC0000302000673B21008E
:1019C000CD0003104C0DF9004D0DFA0079089A3E38
:1019D000CC003F307A3DCD002300920021004C081E
:1019E0002300910020308500223084000230210045
:1019F000D200803120004226883121004808200092
:101A00004202F700210049082000433BF800210072
:101A10004A082000443BF90021004B082000453BC8
:101A2000FA002100CF007908CE007808CD007708B1
:101A3000CC00D501D401D3010A30D2004F08D9001F
:101A40004E08D8004D08D7004C08D6008031200041
:101A5000552688317A08B9007908B8007808B700A7
:101A60007708B6003E084202F7003F08433BF80003
:101A70004008443BF9004108453BFA00BD007908A5
:101A8000BC007808BB007708BA0083103908210031
:101A9000CF00200038082100CE00200037082100A8
:101AA000CD00200036082100CC0020003D08210098
:101AB000D30020003C082100D20020003B08210078
:101AC000D10020003A082100D0008031200081267A
:101AD00088317A082100CF007908CE007808CD003F
:101AE0007708CC00013020006602F7000030673B29
:101AF000FA0077082100D0007A08D100D3010A301B
:101B0000D2005108D5005008D40080312000FB26B7
:101B100088317908FA0078082100CC077908CD3D92
:101B20000030CE3DCF3D20004C08F7004D08F800B6
:101B3000F901FA01CD1F9E2DF903FA0321004C088B
:101B4000F7074D08F83D4E08F93D4F08FA3D780873
:101B50002000CF007708CE005808CE025908CF3BAE
:101B60002100460884004708850020004E088000B8
:101B70004F08813F080021004608FC3E03181A2E3A
:101B8000043E2000242F3930B3000430B40002306A
:101B90002100C9001A2E7130B3000430B4002100B6
:101BA0004808CE004708CD00D0010930CF00803171
:101BB00020005227883179082100CE007808CD0016
:101BC0004E08D2004D08D100D4010530D300803139
:101BD00020001227883179082100C8007808C70042
:101BE000200025080B3C0319FF2D25080F3C031985
:101BF000FF2D20302100C7070030C83D2000210004
:101C0000C81B112E4808023C0318112EFF3A031D71
:101C10000D2E4708E73C0318112E0330C800E730AB
:101C2000C7000230C9001A2EB40103302100C900D8
:101C3000200021004808FA004708C81F272E47083F
:101C4000003CF7000030FA004808FA3B7708CA0069
:101C50007A08CB0010304907840020308500031833
:101C6000850A4B08D2004A08D100D4010A30D300BB
:101C7000803120001227883177082100CF007A08B0
:101C8000D000FA004F088031200021208831F80070
:101C900080002100C91B222F4908003C0318222F75
:101CA000C90B872E4608033C031D872E10304907B9
:101CB0008400203085000318850A4B08D2004A08AA
:101CC000D100D4010A30D30080312000122788319E
:101CD00079082100D0007808CF005008D2004F08C2
:101CE000D100D4010A30D30080312000122788317E
:101CF00077082100CF007A08D000FA004F08803121
:101D000020002120883180388000102F21004B08CE
:101D1000D2004A08D100D4010A30D300803120001B
:101D20001227883179082100CE007808CD00CD082F
:101D3000031DA82ECE08031DA82EC81BA82E1030E8
:101D400049078400203085000318850A8001112F7F
:101D50004B08D2004A08D100D4010A30D3008031A8
:101D600020001227883179082100CE007808CD00A4
:101D7000CD08031DD02ECE08031DD02ECA08031D8A
:101D8000C42ECB080319D02EC81FD02E10304907FF
:101D90008400203085000318850A40308000112F10
:101DA000CA08031DE12ECB08031DE12EC81FE12E3A
:101DB000103049078400203085000318850A80010F
:101DC000112F103049078400203085000318850A40
:101DD0004B08D2004A08D100D4010A30D300803128
:101DE00020001227883179082100D0007808CF0020
:101DF0005008D2004F08D100D4010A30D3008031FE
:101E000020001227883177082100CF007A08D000FF
:101E1000FA004F088031200021208831F80080002E
:101E200021004B08D2004A08D100D4010A30D30067
:101E3000803120001227883179082100CB007808F2
:101E4000CA004A2E200008000A148A140A158207C4
:081E5000C32DCB2D142E142E1E
:102000002508D43E0318EE2A2C3EF02A2D08023C67
:10201000031D1228B001B1015430B2005830B30092
:10202000B401312872087304031926285E082100C0
:10203000C600200051082100C800200050082100DF
:10204000C70088312000BB25903131285E0821006F
:10205000C6007508C8007408C70088312000BB2579
:102060009031EE2A6D30B0007830B1007C30B20093
:102070006E30B300B401EE2A2D08023C031D48283F
:10208000B001B1015430B2005830B300B40153284C
:102090005E082100C6007508C8007408C7008831B2
:1020A0002000BB259031EE2A7C30B0007730B100A3
:1020B0005830B200B300B401EE2A6D30B000793070
:1020C000B1007830B2007C30B300B401EE2A5E0873
:1020D0002100C600200053082100C800200052083B
:1020E0002100C70088312000BB259031EE2A5E30E8
:1020F000B0007930B1003830B2007730B300B401AD
:10210000EE2A54081F3C031D9028D508031D902873
:10211000B0015C30B1007130B200B300B4019F284F
:1021200002302100C600200055082100C800200010
:1021300054082100C70088312000BB259031EE2AC9
:102140007330B0005C30B1007130B200B300B40144
:10215000EE2AD71BBA28D708031DB2285608783CA8
:102160000318BA28B0015C30B1007130B200B3007E
:10217000B401C92802302100C60020005708210000
:10218000C800200056082100C70088312000BB2568
:102190009031EE2A5C30B0007130B1006D30B20089
:1021A0007930B300B401EE2A5E082100C600200099
:1021B00059082100C800200058082100C7008831B4
:1021C0002000BB259031EE2A3E30B0005430B100E3
:1021D0000430B2007830B300B401EE2A5E0821006A
:1021E000C600C801C70188312000BB259031EE2A06
:1021F0006D30B0007830B1007930B2007330B30088
:10220000B401EE2A5E082100C60020005D0821000E
:10221000C80020005C082100C70088312000BB25D1
:102220009031EE2A5E30B0000430B1007730B20059
:102230003D30B300B401EE2A7C30B0007730B100FD
:102240005830B200B300B401EE2A5830B0005C3010
:10225000B1003830B2005E30B300B401EE2A5E083F
:102260002100C60020004D082100C80020004C08B5
:102270002100C70088312000BB259031EE2AB00133
:102280005030B1007930B2007130B300B401EE2AA1
:1022900003302100C60020005B082100C800200098
:1022A0005A082100C70088312000BB259031EE2A52
:1022B0007830B0006E30B1007330B2007930B300C6
:1022C000B401EE2A2D0803196C29013A0319762965
:1022D000033A0319802988292A30B0001530B1004B
:1022E0005030B2007330B300B40188292A30B000F6
:1022F0001530B1005030B2007830B300B4018829F5
:10230000B001B1015430B2005830B300B401882993
:10231000EE2A5030B0007930B100B2005E30B30028
:10232000B401EE2A00302E180130013A03199C291D
:10233000013A0319A629B0295C30B0007330B1000E
:102340007930B2005430B300B401B0295830B00035
:102350003830B1005C30B2006D30B300B401B02948
:10236000EE2A7830B0005830B100B2010630B30028
:10237000B401EE2A5E082100C600200049082100B1
:10238000C800200048082100C70088312000BB2574
:102390009031EE2A7830B0005830B100B2015B3095
:1023A000B300B401EE2A5E082100C60020004B08ED
:1023B0002100C80020004A082100C7008831200001
:1023C000BB259031EE2A5E30B0005830B100B2012A
:1023D0000630B300B401EE2A02302100C600C80165
:1023E0007B08C70088312000BB259031EE2A5E3083
:1023F000B0005830B100B2015B30B300B401EE2A36
:1024000002302100C600C8017E08C70088312000C4
:10241000BB259031EE2A0430B0005E30B100383078
:10242000B2007930B300B401EE2AE108031D202A7E
:10243000B0015C30B1007130B200B300B4012C2A9D
:1024400002302100C600C801200061082100C70039
:1024500088312000BB259031EE2A5E30B000583024
:10246000B1003830B2000430B300B401EE2A5F0886
:10247000323C031D712A2100C501200060082100A3
:10248000C4004508D3004408D200D5016430D4000C
:1024900080312000FB2690317908FA007808B03CA2
:1024A0002100C4000430C5007A08C53B4508C700B8
:1024B0004408C600C9010C30C800803120008227C2
:1024C000903179082100C5007808C4000230C600A8
:1024D0004508C8004408C70088312000BB2590315A
:1024E000A62A60082100C4000A30C500F701F801DF
:1024F000440803104518F707F70CF80CC518F70740
:10250000F70CF80C4519F707F70CF80CC519F70785
:10251000F70CF80C451AF707F70CF80CC51AF70773
:10252000F70CF80C451BF707F70CF80CC51BF70761
:10253000F70CF80C7808643CC4000230C600C801EF
:102540004408C70088312000BB259031EE2A733043
:10255000B0005C30B100B2005030B300B401EE2ADC
:102560002E1DBA2AB001B1015C30B2005430B30064
:10257000B401C12AB0015C30B1007130B200B300C7
:10258000B401EE2A7130B0005030B1007930B200A1
:102590006730B300B401EE2A02302100C600C80142
:1025A00020005F082100C70088312000BB25903142
:1025B000EE2A1C30B0007930B1005030B2006D30DE
:1025C000B300B401EE2A03302100C600C8008E30EB
:1025D000C70088312000BB259031EE2A9031AB2F07
:1025E0000A108A140A11F73E03188A0A8200062884
:1025F0003C28322854285D28672877288128A0287D
:10260000A928CA28D428E428EE28F8280229122963
:102610001C2925292F293F29482958296229892938
:102620009229B129BA29CA29D329E329EC29F72902
:10263000002A0B2A152A2D2A372AA72AB02AC22AAD
:10264000CC2AD92AE32AF030210099000230200058
:10265000A5000430AC00AD012E14AE14AF01B501DD
:10266000B901B801B701B601BD01BC01BB01BA0196
:10267000C101C001BF01BE01C501C401C301C20146
:10268000C701C601C901C801CB01CA01CD0119307A
:10269000CC00CF01CE01E301E201E401E701E60154
:1026A000E901E801E501FF30EA00EB00EF01EE018E
:1026B000ED01EC01F0010330F300E830F200F50128
:1026C000F401F101F601FD01FC012100A101A001CD
:1026D000FB01FE01A301A2012000AE112100A40113
:1026E00023008C018D018E012200920191012000B6
:1026F000A601A7012100A601A501AA01A901A8011F
:10270000A701AE01AD01AC01AB01B201B101B00155
:10271000AF01B601B501B401B301B801B701BA0107
:10272000B901BC01BB01BE01BD01BF01C001411027
:10273000C110C2010830F800063820009C00D030DB
:102740009B0021009114C0308B0407308C00CF30E7
:102750008D0000308E00901124008C01C0308D005F
:1027600021009513083024009000210095132200C9
:102770000D128D122000B40121001E149E141E1192
:10278000073023008C0009308D008A30220097002A
:102790002A0093012200980121001E129E161E138A
:1027A0009E171D14C501C401803120009F25903162
:1027B0007908D1007808D0002100C5010230C4009A
:1027C000803120009F2590317908D3007808D2000D
:1027D0002100C5010430C400803120009F259031C4
:1027E0007908D5007808D4002100C5010630C4005E
:1027F000803120009F2590317908D7007808D600D5
:102800002100C5010830C400803120009F2590318F
:102810007908D9007808D8002100C5010A30C40021
:10282000803120009F2590317908DB007808DA009C
:102830002100C5010C30C400803120009F2590315B
:102840007908DD007808DC000E3023009100951334
:10285000151413082000DE000F302300910095139B
:1028600015141308F80020002E1178182E151030BA
:10287000230091009513151413082000DF00113078
:10288000230091009513151413082000E000123066
:10289000230091009513151413082000E100D11BAB
:1028A000652CD108031D582C5008633C0318652C77
:1028B000D11B692C5108003C0318692CFF3A031DF9
:1028C000652C5008C23C0318692C01302100C2005D
:1028D0002000D31B7F2CD308031D722C5208633CAD
:1028E00003187F2CD31B832C5308003C0318832C24
:1028F000FF3A031D7F2C5208C23C0318832C013081
:102900002100C2002000D51B8E2CD51B922CD5088F
:10291000031D8E2C54081F3C0318922C01302100FB
:10292000C2002000D71B9D2CD71BA12CD708031D4C
:102930009D2C5608823C0318A12C01302100C200B6
:102940002000D91FAD2C5908FF3C031CAD2C031DE2
:10295000B62C5808D73C0318B62CD91BBA2CD9086A
:10296000031DB62C5808283C0318BA2C013021004E
:10297000C2002000DB1BD32C5B08073C031CC62CC9
:10298000031DD32C5A08983C0318D32CDB1BD72CDF
:102990005B08073C0318D72CFF3A031DD32C5A08B9
:1029A000673C0318D72C01302100C20020005C0BCB
:1029B000DC2CDD080319E72C5C08053C031DE32C27
:1029C000DD080319E72C01302100C2002000DE08D9
:1029D0000319F12C5E0BED2CF12C01302100C2000B
:1029E00020005F08323C0319FD2C5F083C3C0319B2
:1029F000FD2C01302100C20020006008023C0318B9
:102A0000052D6008093C0318092D01302100C20082
:102A1000200061084B3C0318112D01302100C20039
:102A200020002100C2080319332D01302000D100FD
:102A30007C30D000D301FA30D200D5010530D4006B
:102A4000D7011E30D600D901D8010830DB00DA01E9
:102A5000DD010530DC00DE012E113230DF000530F3
:102A6000E000E101210020005108E3005008E200ED
:102A70008031C92590318031C92590310A3021003B
:102A8000C40080312000F82D9031AD018031C9257E
:102A9000903122000D128D12FF302000EA00EB0071
:102AA0001A30F700F70B522D000021001E109E1067
:102AB0001E11073023008C0001308D00C73021002B
:102AC0008D0022008D153030F80021001D0883395B
:102AD00078049D000F30F8001F08F03978049F003B
:102AE0000D30F700F70B722D9D149D18752D1C08E5
:102AF000BE001B08BD0022008D11CF3021008D00CB
:102B00001E149E141E11073023008C0009308D0006
:102B1000C3302A0093000830F80021001D088339D3
:102B200078049D000F30F8001F08F03978049F00EA
:102B30000D30F700F70B9A2D9D149D189D2D1B0845
:102B4000B7071C08B83D20002508153C0319AB2D1C
:102B50002A00930120005F08323C031DB92D600854
:102B600076020319B82D0C3060077602031DAF2DD5
:102B7000C22D600876020319C22D0A306007760262
:102B8000031DB92D60087602031DDC2D20302100C5
:102B9000C5005B30C4000130C600803120000E2625
:102BA000903120302100C5005730C400C60180316B
:102BB00020000E269031F42D20302100C500633016
:102BC000C4000130C600803120000E269031203034
:102BD0002100C5005F30C400C601803120000E26F0
:102BE00090312100411420002100C11CFE2D200045
:102BF000AD018031C92590312100C11020002D0880
:102C0000023C031D072E0230C9002B30C800C91F2B
:102C10000C2ED11F182E0E2ED11B1E2E490851022C
:102C2000031C1E2E031D182E5008480203181E2ECA
:102C30007F30EA0022000D16212E2000FF30EA002E
:102C400022002000CB1F272ED11F332E292ED11B6F
:102C50003B2E4B085102031C3B2E031D332E500804
:102C60004A0203183B2E2D0B3B2E7F30EB00220037
:102C70008D163E2E2000FF30EB0022002100BF0AFF
:102C80003F08103C031D7C2E2030C5006730C40077
:102C90002030C7006B30C60088312000E52A903113
:102CA0002100B801B701BC1B5F2EBC08031D5C2EC0
:102CB0003B08823C03185F2EBC011E30BB003B0862
:102CC000B9073C08BA3DC00A4008103C031D7B2EE2
:102CD000C0013A08D2003908D100D4011030D30025
:102CE00080312000122790317908CD007808CC007F
:102CF0002100BA01B901BF01411CC32E33082B07C3
:102D0000C40034082C3DC50035082D3DC6003608EA
:102D10002E3DC7000310470CAE00460CAD00450C1D
:102D2000AC00440CAB002F082707C4003008283D36
:102D3000C5003108293DC60032082A3DC7000310EE
:102D4000470CAA00460CA900450CA800440CA7009B
:102D50002030C5005B30C4002030C7002A30C600D8
:102D6000883120002724903120302100C5005730C1
:102D7000C4002030C7002830C60088312000272436
:102D8000903121004110F1080319E32E2000A5081D
:102D90000319CC2E2100E32EA4018B1BA4178B1347
:102DA0002100ED01EC01200051082100EF0020007E
:102DB00050082100EE008031200032209031A41B09
:102DC0008B17F10121007508CE007408CD00D001E9
:102DD0001E30CF008031200052279031780821002A
:102DE000A5007908A600200049082100CE00200097
:102DF00048082100CD00D0010A30CF0080312000EA
:102E0000522790317908FA00780821002507F80048
:102E10002608FA3D7808A5007A08A6002608C7000B
:102E20002508C600C9012830C8008031200082274B
:102E300090317808F4007908F500500874022100F8
:102E4000C40020005108753B2100C500C51B2F2F71
:102E5000C508031D482F4408023C031C482F740872
:102E6000200050022100C40075082000513B2100C1
:102E7000C500C51B422FC508031D482F4408023C4E
:102E8000031C482F20005108F5005008F4002100D1
:102E90003E08013C031C642F031D522F3D08373CA4
:102EA000031C642F20002E1D582FAD012E14622FFD
:102EB0002D08023C031D612F2100C11420002E109B
:102EC000622F2E10A82F21003E08063C03187E2FEB
:102ED000FF3A031D6F2F3D08063C03187E2F3E0866
:102EE000083C031C7E2F031D792F3D08F93C031C71
:102EF0007E2F2000AD012E14A82F21003E08083C93
:102F00000318992FFF3A031D892F3D08B13C031880
:102F1000992F3E080B3C031C992F031D932F3D084E
:102F2000A43C031C992F01302000AD002E14A82FC3
:102F300021003E080D3C0318A92FFF3A031DA42FC2
:102F40003D08A63C0318A92F02302000AD002E1426
:102F50002100200000285F08323C031DB72FF6082F
:102F60000319B62F76080C3C031DAF2FBE2FF608B1
:102F70000319BE2F76080A3C031DB72F492D6300A5
:107EE00006345734A1345C345D346234FB34673477
:107EF00077346D34F43472344334783474347D34EC
:107F0000833482345C3487341C348C34A63490340B
:107F1000FA3494343034993432349D340B34A134EF
:107F2000BC34A4342E34A8345134AB340E34AE34C3
:107F30004634B03400340034EB340334EC340734CA
:107F400001340C342A34103467341434B734183400
:107F500019341D348C3421340F342634A3342A349C
:107F600045342F34F6343334B534383481343D3429
:107F70005A3442343E3447342D344C342634513450
:107F80002934563435345B344934603464346534D0
:107F900087346A34AF346F34DC3474340F347A3459
:107FA00045347F347E348434BA348934F8348E34A2
:107FB0003734943476349934B5349E34F334A3345E
:107FC0002F34A9346934AE34A034B334D334B83444
:107FD0000234BE342B34C3344F34C8346C34CD3403
:107FE0008134D2348F34D7349434DC348F34E13458
:107FF0008034E6346734EB344234F0341034F534F2
:020000040001F9
:04000E00840FFF1A42
:00000001FF
